:0600000002005B0223CEAA
:03000B000220A12F
:030013000220A127
:03001B0002002BB5
:030023000222F0C6
:10002B0032416C636F726E204D634272696465205E
:10003B00496E632E20536372697074204F53202DC9
:10004B002056657273696F6E20362E30312020205A
:10005B00C2AF75D0007581507A00121D2975B81288
:10006B0075A813787FE4F6D8FD758DFD758BFD753E
:10007B008C88758A0875892175880475368875355D
:10008B00087598C07E007F409020007400F0A3DEBE
:10009B00FCDFFA75A0887800E2F52CD2AFD28CD2B7
:1000AB008E12159290000012207CFAA312207CFB7A
:1000BB00A312207CFCA312207CB46000400274606D
:1000CB00FD4C6018A312207CF540A312207CA312D8
:1000DB00207CF54E90000212156A6017902B40128F
:1000EB001CA37537287455F599780000D8FDD203F9
:1000FB0002019474AAF599780000D8FDC203902BE5
:10010B0051121CA3121C6175382890000F12207C11
:10011B00A2E79209121EAA754520754400754B0083
:10012B00754A30854E4FE54E6056900020A3A3D5FF
:10013B004FFB75A02E7800854E4F12207CF2A30842
:10014B0012207CF2A308B8000205A0D54FEC854E17
:10015B004F854582854483120B85A3A312207C54C3
:10016B000F854B82854A83F0A385824B85834A8515
:10017B004582854483A3A3858245858344D54FD18E
:10018B00121F4D12289D121E507A00121D29D29C4F
:10019B001201BD1202072003F73001F4C201121D38
:1001AB00AE1205F41208BB120A52120BA7120BADBA
:1001BB0080DE12263875D0089021007F4E7E09E034
:1001CB00F5F0A3E0F8A3E0F9686024E5F0547FB400
:1001DB0000051202088018B4010512041C8010B42B
:1001EB0002051202658008B405051205078000E5BB
:1001FB00822406F5820FDEC775D0002222AC83ADB8
:10020B00828F83898275D00075A0247800E0FB75FE
:10021B00F000E425F0F5F00582E5826508602DE03D
:10022B00F208DBEF0582C5F003547FB5F01E858223
:10023B0009902400E0FBA3D20A753803120BF830A7
:10024B000B03121DAE75D0088982800675373C757D
:10025B00D008E5828C838D82F02285820C85830DFC
:10026B00E50FC3944E23245BF50B850F8385098221
:10027B00E030E70FB4F8005007850B82758325F04B
:10028B00020402850B82758325E0B49000400EB406
:10029B00A0004053B4F00302033E020402540FB516
:1002AB0040F8E50904B50803020415850F83F582B0
:1002BB00E030E7030204021582E00509C3943CB465
:1002CB0008005020902400F5F0E540F0A37403F0F3
:1002DB00A3E5F0F075D0007BFF902400D20A120B3F
:1002EB00F875D008020402540FB540AEE50904B509
:1002FB000803020415850F83F582E030E70302043F
:10030B000260B41582E00509C3943CB40800502088
:10031B00902400F5F0E540F0A37402F0A3E5F0F0B3
:10032B0075D0007BFF902400D20A120BF875D00811
:10033B00020402E508C39509B4090050030203E95E
:10034B00850F83850982E0B47F7F0582E0B47F024D
:10035B008003B540740582E0B4026E0582E0B47F81
:10036B00028008B410028003B4305E0582E0B40151
:10037B00580582E020E752C3943075F00AA4F5F0DB
:10038B000582E020E743C3943025F075F00AA4F50D
:10039B00F00582E020E732C3943025F0F5F00582BA
:1003AB00E0B4F725858209902400E540F0A374188A
:1003BB00F0A3E5F014F075D0007BFF902400D20A77
:1003CB00120BF875D00802040230E7030203FD7527
:1003DB00373C850B8275832574F7F0020402850F79
:1003EB0083850982E020E70A0582E582B508F502DC
:1003FB0004158582091509850C82850D83E5090491
:10040B00F0F50965086003020275850C82850D8382
:10041B0022AC83AD8275D010E508B509030204A5A3
:10042B00850F83850982E00509B4F5ECA809150948
:10043B00E508C398B4050050030204A51204B0B537
:10044B004045902400F0A3F5F01204B0FBB4030078
:10045B00503525F0F5F01204B0602CB44000502755
:10046B00F925F0F5F0E92405FAE508C39509FEB581
:10047B00120040261204B0F0A325F0F5F0D9F512C6
:10048B0004B0B5F002800875373C050902042375EA
:10049B0038031204C0880902042375D008E5098CBF
:1004AB00838D82F022C083C082850F838882E0080F
:1004BB00D082D0832275D0007BFF902400D20A1209
:1004CB000BF8E513B40002802FB40214E50FC394AC
:1004DB004EFA850F83850982E516FBD20A121D336E
:1004EB00E50FC3944EFA74AA30120274559024008F
:1004FB00F07B01D20A121D3375D01022AC83AD8272
:10050B0075D010A809E508C398B40C004073120508
:10051B0097B4180050641204B0B43A5E120597B445
:10052B003C0050561204B0B43A50120597B43C003C
:10053B0050481204B0B420421204B0B4203C120450
:10054B00B0B420361204B0B40D30753803902400CB
:10055B00A809791C1205971205C708791D12059772
:10056B001205C708791E1205971205C7791FE412E9
:10057B0005C7080808088809808975373C05098074
:10058B008275D008E5098C838D82F022C083C082EE
:10059B00850F838882E0080582C39430B40600502F
:1005AB001475F00AA4F5F0E008C39430B40A0050B7
:1005BB000425F0800274FFD082D08322C0F0F5F0C6
:1005CB00E540F0A37428F0A3E9F0A3E5F0F0A32431
:1005DB00282903547FF075D0007BFF902400D20AAA
:1005EB00120BF875D010D0F022908800E0F8C52CD3
:1005FB006830E00CC0E0A26075F000120671D0E02C
:10060B0030E10CC0E0A26175F001120671D0E03050
:10061B00E20CC0E0A26275F002120671D0E030E38A
:10062B000CC0E0A26375F003120671D0E030E40C4D
:10063B00C0E0A26475F004120671D0E030E50CC086
:10064B00E0A26575F005120671D0E030E60CC0E053
:10065B00A26675F006120671D0E030E708A2677546
:10066B00F00712067122920590257DE070030207B8
:10067B00D3F54F754D00754C26854D82854C83E027
:10068B00F9A3E0FAA3E0A3A385824D85834C89826D
:10069B008A83F545C0F075F002A4F54B85F04AD07E
:1006AB00F0A3A312207CFBA312207CFCA312207CC2
:1006BB00FDA312207CFEA312207CFFEF547FB5F02C
:1006CB005EEB20E4052005578003300552EE600CED
:1006DB00B4070050071207D740028043903000E563
:1006EB00452582F582E030E23030E02FE54B2400E7
:1006FB00F582E54A3431F583120B98E582C39CE50C
:10070B00839D50030207D0E5451212E975833085AE
:10071B004582E0D2E2F00207D0D2E2F00207D0A38A
:10072B0012207CFEA312207CFFEF547FB5F02BEB45
:10073B0020E505200524800330051FEE600CB4076F
:10074B000050071207D740028010903000E5452576
:10075B0082F582E0C2E2F00207D0A312207CFEA356
:10076B0012207CFFEF547FB5F02BEB20E605200524
:10077B0024800330051FEE600CB4070050071207EE
:10078B00D740028010903000E5452582F582E0D2FB
:10079B00E3F00207D0A312207CFEA312207CFFEF14
:1007AB00547FB5F020EB20E70520051980033005B9
:1007BB0014EE600CB4070050071207D740028005F7
:1007CB00E5451212E9D54F0122020684C082C0838F
:1007DB00C0F0E5822407F582E5833400F58312200F
:1007EB007CF8A312207C541F240BF975A025E3F988
:1007FB00EE30E708E8541F240BF8E2F8EE540F2311
:10080B00239008107302085000020854000208627B
:10081B00000208700002088000020892000208A281
:10082B0000020854000208620002087000020880EF
:10083B0000020892000208A20002085000020850B1
:10084B000002085000C30208B4E988F0B5F004D3E5
:10085B000208B4C30208B4E988F0B5F004C3020877
:10086B00B4D30208B4E988F0B5F0004004C3020821
:10087B00B4D30208B4E988F0B5F00280064004C393
:10088B000208B4D30208B4E889F0B5F00040E2C323
:10089B000208B4D30208B4E889F0B5F00280064030
:1008AB0004C30208B4D30208B4D0F0D083D08222A0
:1008BB00200F030209EA90257EE070030209EAF596
:1008CB004F754D00754C2A854D82854C83E0F9A3FD
:1008DB00E0FAA3E0A3A385824D85834C89828A83AA
:1008EB00F545C0F075F002A4F54B85F04AD0F0A3A6
:1008FB00A312207CFBA312207CFCA312207CFDA363
:10090B0012207CFEA312207CFFEE541FB407004084
:10091B004A1209ED40028043903000E5452582F5EF
:10092B0082E030E23030E02FE54B2400F582E54ADF
:10093B003431F583120B98E582C39CE5839D5003FC
:10094B000209D6E5451212E9758330854582E0D25E
:10095B00E2F00209D6D2E2F00209D6A312207CFE05
:10096B00A312207CFFEE541FB4070040171209EDB1
:10097B0040028010903000E5452582F582E0C2E20E
:10098B00F00209D6A312207CFEA312207CFFEE54AA
:10099B001FB4070040171209ED4002801090300081
:1009AB00E5452582F582E0D2E3F00209D6A31220B9
:1009BB007CFEA312207CFFEE541FB40700400C12E8
:1009CB0009ED40028005E5451212E9D54F030209F6
:1009DB00DF0208D27E2090252B7400F0A3DEFCC230
:1009EB000F22C082C083C0F0E5822407F582E58325
:1009FB003400F58312207CF8A312207C541FF9904D
:100A0B00252B2582F582E0C2046002D204EE30E78A
:100A1B0019E8541FF890252B2582F582E06002D24D
:100A2B000475A025740B28F8E2F830041275A02584
:100A3B00740B29F9E3F9EE540F232390081073C3B9
:100A4B00D0F0D083D08222854E4FE54E7003020B3F
:100A5B0049754B00754A30754D00754C2E90002032
:100A6B00E54E120B4A8582478583467543007542D6
:100A7B0031854B82854A83E020E203020B0A8543D2
:100A8B0082854283120B98A38542A0A843E582F28C
:100A9B0008E583F2854D82854C83120B988582493C
:100AAB00858348120B85E58245836019120B5D60C7
:100ABB0041A3A3C20A120BF8200637854982854849
:100ACB0083A3A380D8854782854683120B858582B5
:100ADB00498583488542A0A8437400F208F2854BF0
:100AEB0082854A83E030E10510E3028002C2E2C254
:100AFB00E4F0854D82854C83E549F0A3E548F0D5BC
:100B0B004F02803A854B82854A83A385824B85832E
:100B1B004A854D82854C83A3A385824D85834C8565
:100B2B004782854683A3A385824785834685438277
:100B3B00854283A3A3858243858342020A7C22C01C
:100B4B00F075F002A42582F582E5F03583F583D0AC
:100B5B00F022AD82AE83120B85AB82AC83854382D0
:100B6B00854283120B98E582C39BE5839C400474FA
:100B7B00FF800274008D828E8322C0F012207CF5E0
:100B8B00F0A312207CF58385F082D0F022C0F0E038
:100B9B00F5F0A3E0F58385F082D0F022AA24121D94
:100BAB002922301347E550B4024214F550780075F2
:100BBB00A02574FFF208E540F2087400F208E52C5A
:100BCB00F208E52DF208E52EF208E52FF2089080E9
:100BDB0000E0F208A3A3E0F208A3A3E0F208E4F21A
:100BEB0008F29025007A007B2B121D3322C206AD32
:100BFB0082AE837A00122088FFA3122088C212B41F
:100C0B0050004003D21222902A6075F002A4258274
:100C1B00F582E5F03583F583E493F5F0A3E4938552
:100C2B00F083F582E473120D53020D4E120D9502F3
:100C3B000D4E120DD6020D4E120E16020D4E120E49
:100C4B005C020D4E120E9E020D4E120EAF020D4E99
:100C5B00120EE0020D4E120EF8020D4E120F210273
:100C6B000D4E121078020D4E1210D6020D4E1211AF
:100C7B00EB020D4E121200020D4E121245020D4EDA
:100C8B0012128A020D4E1212A3020D4E1212BC0248
:100C9B000D4E1212D5020D4E1213DF020D4E121411
:100CAB00F0020D4E121715020D4E020D4E121C6165
:100CBB00020D4E121C81020D4E12176B020D4E12BD
:100CCB001799020D4E1217FD020D4E121821020D2F
:100CDB004E12184D020D4E12187A020D4E1218AB11
:100CEB00020D4E1218DA020D4E12190D020D4E1294
:100CFB00193E020D4E121965020D4E12198E020D80
:100D0B004E1219BA020D4E1219EB020D4E121A1E8B
:100D1B00020D4E121A55020D4E121A8A020D4E1268
:100D2B001AC3020D4E121AFA020D4E121B29020D96
:100D3B004E1217C7020D4E121B5A020D4E121C4BB0
:100D4B00020D4E8D828E83228D828E83A3A3122061
:100D5B008820E629121550B900104224F4F5F090C2
:100D6B002040E055F0F05228801FB901104225F4C5
:100D7B00F5F0902041E055F0F05229800C543F24BF
:100D8B0074F58275832074FFF0228D828E83A3A36A
:100D9B0012208820E628121550F4B9000F5224F5C2
:100DAB00F0902040E055F0F05228801EB9010F5210
:100DBB0025F5F0902041E055F0F05229800C543F7E
:100DCB002474F5827583207400F0228D828E83A3A8
:100DDB00A3122088F8541F232400C8121550FAA31D
:100DEB0012208875A020F208F2EAB9000DF5F090F8
:100DFB002040E045F0F042288010B9010DF5F0904D
:100E0B002041E045F0F042298000228D828E83A3A1
:100E1B00A3122088F8541F232400C8121550FAA3DC
:100E2B0012208875A020F208F2EAB900104228625D
:100E3B0024F4F5F0902040E055F0F08013B9011048
:100E4B0042296225F4F5F0902041E055F0F0800046
:100E5B00228D828E83A3A312208820E6291215509F
:100E6B00B900106224F4F5F0902040E055F0F052F8
:100E7B0028801FB901106225F4F5F0902041E05550
:100E8B00F0F05229800C543F2474F582758320E0D6
:100E9B00F4F0228D828E83A3A3122088543FFBA3F0
:100EAB001215F022902200E0F8A3E0F5F075A057A0
:100EBB00902B007900E993600BF20908E8B5F0F587
:100ECB00D2068010902200E8C2ACF0200804D208B1
:100EDB00D299D2AC228D828E83A3A3122088FAA33F
:100EEB00122088FBA3121D336002D206228D828E44
:100EFB0083A3A3122088FA7B01A312208890250BD1
:100F0B002582F582A20AC0D0D20A121D33D0D0920C
:100F1B000A6002D206228D828E83A3A3122088FA46
:100F2B00A3122088C0E0A3122088FF54072323902C
:100F3B000F3E73020F5D00020F8F00020FBA00020B
:100F4B000FDF00020F5D00020F5D00020F5D00025C
:100F5B000F5DD0E090250B2582F582E078007900BB
:100F6B007C00600F75F00A84A8F0600775F00A84A6
:100F7B00A9F0FCE82430F8E92430F9EC2430FC7BB0
:100F8B0003020FFDD0E090250B2582F582E0540F74
:100F9B002430B43A0040022407F9E054F0C4243062
:100FAB00B43A0040022407FC78207B02020FFDD0EC
:100FBB00E090250B2582F582E054072430F8E054AD
:100FCB00380303032430F9E054C023232430FC7B83
:100FDB0003020FFDD0E090250B2582F5827B01A249
:100FEB000AC0D0D20A121D33D0D0920A607ED2062C
:100FFB00807AEF543803901005730210240002100E
:10100B005800021049000210320002102400021096
:10101B00240002102400021024BB0102802FBC30DC
:10102B002CE9FCE8F9DBF2BC3023E9FCE8F9782089
:10103B00BB031ABC3017E9FCE8F97820800FBC30F1
:10104B000C7C20BB0307B93004792080009020442E
:10105B00ECF0A3E9F0A3E8F0902044A20AC0D0D2B0
:10106B000A121D33D0D0920A6002D206228D828ED4
:10107B0083A3A3122088FAA3122088F8A312208836
:10108B00F9A312208890250B2582F582E0FB902096
:10109B00447406F0A3E5404480F0FCA3E8F02CFC7C
:1010AB00A37428F02CFCA3E9F02CFCA3EBF02CA3ED
:1010BB0003547FF09020447B07A20AC0D0D20A12BF
:1010CB001D33D0D0920A6002D20622854B82854A0C
:1010DB0083E0F98D828E83A3A3122088FA23232326
:1010EB00FC75A021F8E920E442E2C2E7F2E408F241
:1010FB0008F2A3122088FBA3121D3375A021ECF874
:10110B00E2D2E7F20808080808122088F2A30812B6
:10111B002088F2200606A308122088F2854B8285D0
:10112B004A83E0D2E4F0D2060211EA08A312208827
:10113B0024052582F582E43583F583122088F5F0AA
:10114B00E2C395F0501E08080808E2F5F008E245E6
:10115B00F0602D18E2C39401F2500408E214F2D2AD
:10116B00060211EAABF0A3EA244EF5A07800122098
:10117B0088F5F0E2B5F009A308DBF3753803804A74
:10118B0075A021EC2407F8E2600F14F28D828E8398
:10119B00A3A3ECF8D2060210F475373C30092B9060
:1011AB00001412207CF8A312207CF5838882E58240
:1011BB002AF582E43583F58312207CF8C3954E50D3
:1011CB00097583308882E0D2E2F075A021ECF8E259
:1011DB00C2E7F2854B82854A83E0C2E4F0C2062265
:1011EB008D828E83A3A3122088547F232549F54932
:1011FB0050020548228D828E83A3A312208820E7FC
:10120B001810E60A121550B90004782480172474BC
:10121B00F875A020E270138020547F121550B9008E
:10122B0004782C8000567002800FA3122088547F04
:10123B00232549F54950020548228D828E83A3A3AD
:10124B0012208820E71810E60A121550B90004780E
:10125B002480172474F875A020E260138020547F3B
:10126B00121550B90004782C8000566002800FA331
:10127B00122088547F232549F54950020548228DB9
:10128B00828E83A3A3122088F8C3954E50097583D1
:10129B00308882E0D2E2F0228D828E83A3A31220CB
:1012AB0088F8C3954E50097583308882E0C2E2F00E
:1012BB00228D828E83A3A3122088F8C3954E5009EA
:1012CB007583308882E0D2E3F0228D828E83A3A3D4
:1012DB00122088F8C3954E5004E81212E922C00080
:1012EB00C003C004C0F0F8900020E54E120B4AE892
:1012FB00120B4A120B85AB82AC8375832EE875F00B
:10130B0002A4F582E5F03583F583EBF0A3ECF075E1
:10131B008331E875F002A4F582E5F03583F583E4BB
:10132B00F0A3F07583308882E0C2E2C2E4F0C2E33E
:10133B00D0F0D004D003D00022902200E0F875A0AA
:10134B00577402F20890000212207CA3F2081220BC
:10135B007CF208902200E8C2ACF0200804D208D23C
:10136B0099D2AC22C004C005C00675A025784B7974
:10137B0010750400750500750604D5041DD5051AF6
:10138B00D506177455C29BC299F59975040075055E
:10139B0004D504FDD505FA02005B3098DDE599F222
:1013AB00C298DA04EB60121B08D9C6784B7910E2AD
:1013BB0012206CA308D9F880B17A007B20DAFEDB0F
:1013CB00FC784B7910E212206CA308D9F8D006D028
:1013DB0005D00422C2AF8D828E83A3A3122088FA7C
:1013EB00A3122088FBE599C29874AAC29BC299F5F7
:1013FB009990000012136F02005B8D828E83A3A362
:10140B00122088FAA3122088FB90000212207CF88D
:10141B00A312207CC854F0241CC8500104F5838807
:10142B0082745A12206CA374A512206CA3EA1220AA
:10143B006CA3EB12206CA3C000C0017500007501FA
:10144B0000D500FDD501FAD001D000C2AFE599C29D
:10145B009874AAC29BC299F59912136F74AAC29B76
:10146B00C299F599750400750504D504FDD505FAE7
:10147B0002005B2014FDC29BD214F599229000024E
:10148B0012207CF8A312207CC854F0241CC85001F5
:10149B0004F583888212207CB45A18A312207CB4E2
:1014AB00A511A312207CFAA312207CFBA3BA000C7B
:1014BB00BB0009E412147E12147E801AEA12147E09
:1014CB00EB12147E12207CA312147E1ABAFF011B9E
:1014DB00BA00F1BB00EE750400750504D504FDD50B
:1014EB0005FA02005B90000212207CFAA312207C0A
:1014FB00FB700CEA7009E412147E12147E80278AAA
:10150B00828B83A3A3AA82AB83EA12147EEB121401
:10151B007E90000012207CA312147E1ABAFF011BCE
:10152B00BA00F1BB00EE750400750504D504FDD5BA
:10153B0005FA02005B8D828E83A3A3122088C2134F
:10154B006002D21322F95407C90303035403C0E00A
:10155B007401B90002800323D9FDF9D0E0C92278C8
:10156B0000790012207C28500109F8A3DC05BD008E
:10157B00F28006BCFFED1D80EAE86A7007E96B702C
:10158B0003E4800274FF2290000075A0987802E2B9
:10159B0030E70BA3E583B405F6C2110215EFD211A8
:1015AB007A30121CC77A30121CC77A38121CC77AD1
:1015BB0080121CC77A06121CC77A0C121CC77A0140
:1015CB00121CC77A40121CC77A5A121CE67A4012B8
:1015DB001CC7121D08B45AC1902B2F121CA3902BA1
:1015EB0015121CB5227A80121CC7122088B4040075
:1015FB005029A3DB028050B400047A808010B40120
:10160B00047AC08009B402047A9480027AD412203E
:10161B0088A3543F2AFA121CC7802AB40C08A37A59
:10162B0001121CC7801FB40D03A38014B40A03A3BB
:10163B00800EB40E2EDB11800EFA121CE6A3800571
:10164B007AC0121CC7DBA322A312208814A3C0826A
:10165B00C08390250B2582F582E0D083D0821216B1
:10166B00D180E2B40FD3DB0280DDA312208814A358
:10167B00C082C08390250B2582F582E0D083D08277
:10168B0012169080C07C017A20C39464400C1C7AA3
:10169B0031C394644004C394640A2464C0E0121CF4
:1016AB00E6D0E07A31C3940A40030A80F81A240A80
:1016BB00C0E0BA3005EC60027A20121CE6D0E024C0
:1016CB0030FA121CE6227C017A20C39464400C1C75
:1016DB007A31C394644004C394640A2464BA20022C
:1016EB008007C0E0121CE6D0E07A31C3940A4003B5
:1016FB000A80F81A240AC0E0BA3003EC7003121CFB
:10170B00E6D0E02430FA121CE6228D828E83A3A34E
:10171B001220885403FB7005902B628013B40105D3
:10172B00902B72800BB40205902B828003902B922E
:10173B007A01121CC77C10E493FA121CE6A3DCF7A7
:10174B007C107AC0121CC7EBC42474F582758320FD
:10175B00E060047A3180027A30121CE6A3DCF122BD
:10176B008D828E83A3A3122088FAA3122088FBEA12
:10177B004224F4F5F0902040E055F0F05228EB4273
:10178B0025F4F5F0902041E055F0F05229228D829E
:10179B008E83A3A3122088FAA3122088FBEAF452AB
:1017AB0024F5F0902040E055F0F05228EBF4522550
:1017BB00F5F0902041E055F0F05229228D828E8376
:1017CB00A3A3122088FAA3122088FBEA7011EBF571
:1017DB0024F4F5F0902040E055F0F052288012B43C
:1017EB00010FEBF525F4F5F0902041E055F0F052A8
:1017FB0029228D828E83A3A3122088541FF9240BD8
:10180B00F8A312208875A025F275A025742B29F852
:10181B0074FFF2D20F228D828E83A3A312208854E1
:10182B001FF9240BF875A025E2F5F0A3122088B55B
:10183B00F00FA3122088547F232549F54950020548
:10184B0048228D828E83A3A3122088541F240BF869
:10185B0075A025E2F5F0A3122088B5F002800FA346
:10186B00122088547F232549F54950020548228DC3
:10187B00828E83A3A3122088541F240BF875A025F6
:10188B00E2F5F0A3122088C5F0B5F0004002800FFE
:10189B00A3122088547F232549F54950020548227D
:1018AB008D828E83A3A3122088541F240BF875A05E
:1018BB0025E2F5F0A3122088B5F0004002800FA3BB
:1018CB00122088547F232549F54950020548228D63
:1018DB00828E83A3A3122088541F240BF875A02596
:1018EB00E2F5F0A3122088C5F0B5F00280044002A7
:1018FB00800FA3122088547F232549F549500205F8
:10190B0048228D828E83A3A3122088541F240BF8A8
:10191B0075A025E2F5F0A3122088B5F002800440F3
:10192B0002800FA3122088547F232549F5495002CA
:10193B000548228D828E83A3A3122088541FF9247D
:10194B000BF875A025E2FAA31220882AF275A025C0
:10195B00742B29F974FFF3D20F228D828E83A3A3EC
:10196B00122088541FF9240BF875A025E2FAA31254
:10197B002088CAC39AF275A025742B29F974FFF33A
:10198B00D20F228D828E83A3A3122088541FF5F0D1
:10199B00240BF8A3122088541F240BF975A025E300
:1019AB00F275A025742B25F0F874FFF2D20F228D5F
:1019BB00828E83A3A3122088541F240BF875A025B5
:1019CB00E2F5F0A3122088541F240BF9E3B5F00FB6
:1019DB00A3122088547F232549F54950020548223C
:1019EB008D828E83A3A3122088541F240BF875A01D
:1019FB0025E2F5F0A3122088541F240BF9E3B5F070
:101A0B000280DCA3122088547F232549F54950021C
:101A1B000548228D828E83A3A3122088541F240B8A
:101A2B00F875A025E2F5F0A3122088541F240BF9BA
:101A3B00E3C5F0B5F0004002800FA3122088547F5D
:101A4B00232549F54950020548228D828E83A3A395
:101A5B00122088541F240BF875A025E2F5F0A31271
:101A6B002088541F240BF9E3B5F0004002800FA32C
:101A7B00122088547F232549F54950020548228DB1
:101A8B00828E83A3A3122088541F240BF875A025E4
:101A9B00E2F5F0A3122088541F240BF9E3C5F0B52F
:101AAB00F00280044002800FA3122088547F23256C
:101ABB0049F54950020548228D828E83A3A312203B
:101ACB0088541F240BF875A025E2F5F0A31220888B
:101ADB00541F240BF9E3B5F00280044002800FA3DE
:101AEB00122088547F232549F54950020548228D41
:101AFB00828E83A3A3122088541FF5F0240BF87554
:101B0B00A025E2FAA3122088541F240BF9E32AF232
:101B1B0075A025742B25F0F874FFF2D20F228D825D
:101B2B008E83A3A3122088541FF5F0240BF875A005
:101B3B0025E2FAA3122088541F240BF9E3CAC39A97
:101B4B00F275A025742B25F0F874FFF2D20F228DBD
:101B5B00828E83A3A3122088541FF9902BA27A01A3
:101B6B00121CC77C10E493FA121CE6A3DCF77AC0B4
:101B7B00121CC79024007420F0A3F0A3F0A3F0A3D1
:101B8B00E904121BE3EBB430027420F0A3EAF0A3D8
:101B9B007420F0A3743DF0A37420F0A375A025E985
:101BAB00240BF9E3121BE3ECD204B43004C204742B
:101BBB0020F0A3EBB430052004027420F0A3EAF06C
:101BCB00A37420F0A3F0A3F0A3F07C10902400E00A
:101BDB00FA121CE6A3DCF8227A007B007C0060166C
:101BEB0075F00A84AAF0600E75F00A84ABF06006FB
:101BFB0075F00A84ACF0EA2430FAEB2430FBEC24C9
:101C0B0030FC2290000012207CFB90200012207CE4
:101C1B00FDEBF412206C121C5612207CF4B5030E53
:101C2B0090000012207CB503057A18021C3B7A0841
:101C3B00902000ED12206C121C5690257FEAF022AA
:101C4B00121C0E90257FE0FAF599227C0075F01995
:101C5B00DCFED5F0FB227A80121CC77B28902580F6
:101C6B00121D08F0A3DBF97AC0121CC77B28121DCA
:101C7B0008F0A3DBF9227A80121CC77B2890258001
:101C8B00E0FA121CE6A3DBF87AC0121CC77B28E033
:101C9B00FA121CE6A3DBF8227A80121CC77400939D
:101CAB006007FA121CE6A380F4227AC0121CC774D8
:101CBB0000936007FA121CE6A380F422C0F03011E7
:101CCB001775F00075A0987802E230E70700D5F0A1
:101CDB00F3021CE37800EAF2D0F022C0F030111AC4
:101CEB0075F00075A0987802E230E70700D5F0F3A5
:101CFB00021D0575A0987801EAF2D0F022C0F030F1
:101D0B00111975F00075A0987802E230E70700D53D
:101D1B00F0F3021D2675A0987803E2D0F02275A08F
:101D2B00807800EAF4F22222AE82AF83902200EA9E
:101D3B002323232582F58274003583F583E0F8A3F2
:101D4B00E0F9EA2457F5A089F08E828F8312208860
:101D5B00F2A308E8B5F003021DA7DBF1AE82AF8357
:101D6B00902200EA2323232582F58274003583F524
:101D7B0083E8BA000FC2ACF0200804D208D299D283
:101D8B00AC021DA1D20BF0902064EA14540F2582F3
:101D9B00F582E0D2E7F0E48E828F832274FF8E828D
:101DAB008F8322200B03021E4F90001212207CF512
:101DBB00F0A312207CF58385F082A3E5822411F534
:101DCB0082E5833400F583AE82AF8390206475A0E7
:101DDB00907A00C082C0838E828F8312207C54E065
:101DEB00B4E007D083D082021E37D083D082E0309C
:101DFB00E73AC2E7F0EAC4032402F8C082C0838E3C
:101E0B00828F8312207CB40A168FF07465F27FD711
:101E1B00C2AFDFFE7475F27F24DFFED2AFAFF0D01E
:101E2B0083D08274A5F20808087406F2A3C082C09E
:101E3B00838E828F83A3AE82AF83D083D0820ABA84
:101E4B000891C20B2290000A12207C6016758C0040
:101E5B00758A00D2A9D2AA7530FFF534853433D2F6
:101E6B00078039C20790000912207CB40008753630
:101E7B006A753508801CB401087536877535E9809D
:101E8B0011B403087536707535088006753688757C
:101E9B00350885368C85358AC2AAD2A9D20222E5AD
:101EAB004E7003021F4C854E4F7A007B00780079F1
:101EBB002A7D0075F0267545207544008545828581
:101ECB004483120B85AE82AF8374052582F5827431
:101EDB00003583F5837C04C204C20512207CA36009
:101EEB0002D20412207CA3B4FF028002D205DCEBE9
:101EFB0030041788828983EEF0A3EFF0A3E54EC37D
:101F0B00954FF0A3A3A882A9830B3005198D828569
:101F1B00F083EEF0A3EFF0A3E54EC3954FF0A3A330
:101F2B00AD828583F00A854582854483A3A3858290
:101F3B0045858344D54F8590257EEBF090257DEA32
:101F4B00F022C2A878087A007B0890001212207C3D
:101F5B00F5F0A312207CF58385F082A312207CF58B
:101F6B0023A3AE82AF83E5822410F582E583340090
:101F7B00F58312207CFD75A021BD00067400D2E70D
:101F8B008043BD05067402D2E7803ABD0606740293
:101F9B00D2E78031BD0C067401D2E78028BDE00684
:101FAB007404D2E7801FBD0D067405D2E78016BD01
:101FBB000E067407C2E7800DBD0F067406D2E780CC
:101FCB00047403C2E7F2FCE82402F975A022ECF3D7
:101FDB00BDE00302204E75A090EA2400F9090974B4
:101FEB0010F319197402A21EB392E0BD0002800314
:101FFB00BD0E0444188011A21BB392E4A21C92E202
:10200B00A21D5004C2E4D2E3F37407301F02740F15
:10201B00F3EA2401F9902064E5235407FC93F3EAD7
:10202B002404F97488BC06028008BD05028003BD38
:10203B0006027408F3EA2402F97401F3EA2405F9A1
:10204B007404F38F838E82E82408F8EA2408FADB01
:10205B00028003021F67D2A82244668899BBCCCCAE
:10206B00BBC083C0E0E58324A0F583D0E0F0D08330
:10207B0022C083E58324A0F583E0D08322300D04B6
:10208B00E4938011300A03E0800BC083E58324A026
:10209B00F583E0D08322C0D0C0E0C083C08275D06E
:1020AB0010D55003755010E538B40004D2B4800439
:1020BB001538C2B4E537B40004D2B580041537C265
:1020CB00B5300005D54102C200E52870030221CBD3
:1020DB0030401B902001E014F07013C240B22090EE
:1020EB002040E030E008902000E0A3F0D2403041E7
:1020FB001B902003E014F07013C241B221902040DA
:10210B00E030E108902002E0A3F0D24130421B9076
:10211B002005E014F07013C242B222902040E03050
:10212B00E208902004E0A3F0D24230431B9020073A
:10213B00E014F07013C243B223902040E030E30868
:10214B00902006E0A3F0D24330441B902009E0140A
:10215B00F07013C244B224902040E030E408902089
:10216B0008E0A3F0D24430451B90200BE014F07034
:10217B0013C245B225902040E030E50890200AE0DC
:10218B00A3F0D24530461B90200DE014F07013C223
:10219B0046B226902040E030E60890200CE0A3F0F9
:1021AB00D24630472290200FE014F0701AC247B28B
:1021BB0027902040E030E70F90200EE0A3F0D247AD
:1021CB00E52970030222C230481B902011E014F065
:1021DB007013C248B228902041E030E008902010E4
:1021EB00E0A3F0D24830491B902013E014F0701399
:1021FB00C249B229902041E030E108902012E0A3BF
:10220B00F0D249304A1B902015E014F07013C24AEB
:10221B00B22A902041E030E208902014E0A3F0D2E3
:10222B004A304B1B902017E014F07013C24BB22BAB
:10223B00902041E030E308902016E0A3F0D24B3021
:10224B004C1B902019E014F07013C24CB22C902050
:10225B0041E030E408902018E0A3F0D24C304D1B45
:10226B0090201BE014F07013C24DB22D902041E072
:10227B0030E50890201AE0A3F0D24D304E1B902091
:10228B001DE014F07013C24EB22E902041E030E6E8
:10229B000890201CE0A3F0D24E304F1B90201FE083
:1022AB0014F07013C24FB22F902041E030E708902A
:1022BB00201EE0A3F0D24F30020FD201853E838562
:1022CB003F82A385833E85823F200710C28CE58A1F
:1022DB002535F58AE58C3536F58CD28CD082D083BA
:1022EB00D0E0D0D032C0D0C0E0C083C08275D0184F
:1022FB0020980F309903022366D082D083D0E0D090
:10230B00D032C298902101E0F8A3E0F9A3E0FAA340
:10231B00E0FBE599FF309A1030E70DC29A7B01E89C
:10232B00FA0AEA6970027B00EB602175834E8A82A0
:10233B00EFF00582E5826970047B00800FAA820BA7
:10234B00309A098882EB14F0EAF87B00902101E8BF
:10235B00F0A3A3EAF0A3EBF00222FBC299101490B6
:10236B00902200E0F8A3E0B5180CE4902203F0A350
:10237B00F0C2080222FBF8902204E070127583571A
:10238B008882E0902203F0902201E004F08011F8A3
:10239B00902203E014B5180CE4902203F0A314F080
:1023AB00D29B8002C29B902201E0758357F582E09D
:1023BB00F5990582E582902201F0A3A3A3E004F036
:1023CB000222FBC0D0C0E0C0F0C083C08275D01821
:1023DB00753C08753D00753B0090001212207CF592
:1023EB00F0A312207CF58385F082E53D2412258233
:1023FB00F582E5833400F58312207CB4E0030226DA
:10240B001DE53B9090052582F582E020E203022436
:10241B00E0C0E0902108E53B2582F582E0FCA38536
:10242B00823A858339547FB4000E909001E53B25A9
:10243B0082F582E0A2E5920C909003E53B2582F5B4
:10244B0082E0F5F0EC20E7030224DE547FB40003B6
:10245B0002247E853A82853983E0F582E53D244F5F
:10246B00F583E5F0F00582E582853A82853983F0C4
:10247B000224DE853A82853983E0FCA3E0FDA3E0EC
:10248B00FEA3E0FFE5F0300C1030E70DC20C7F012E
:10249B00ECFE0EEE6D70027F00EF60258E82E53D47
:1024AB00244FF583E5F0F00582E5826D70047F0023
:1024BB00800FAE820F300C098C82EF14F0EEFC7F94
:1024CB0000902109E53B2582F582ECF0A3A3EEF009
:1024DB00A3EFF0D0E020E00302261D902208E53D9B
:1024EB002323232582F582E0FFA3E0B51F22A3A3BC
:1024FB007400F0A3F0909002E53B2582F58274B155
:10250B00F0909005E53B2582F5827404F002261DC0
:10251B00F5F085823A858339A3E0547FB4000280BD
:10252B0008B4070280030225F9C0E0A3E0FC6001B8
:10253B0014FEA3E0FDD0E0B40705BC00538003BC40
:10254B00001FE5F0F582E53D2458F583E0FC05829C
:10255B00E582853A82853983F0F5F0B51F070224B1
:10256B00F9EDB51E2B909002E53B2582F582741593
:10257B00F0909000E53B2582F582E0FEA3A3741555
:10258B00F0909000E53B2582F582EE4404F0802923
:10259B00909002E53B2582F5827415F0909000E552
:1025AB003B2582F582E0FEA3A37415F0909000E525
:1025BB003B2582F582EE54FBF0E5F0F582E53D24F8
:1025CB0058F583E0FE0582E582853A82853983F0F2
:1025DB000DECB51D047C007D00A3A3ECF0A3EDF086
:1025EB00909003E53B2582F582EEF002261DE5F087
:1025FB00F582E53D2458F583E0F5F00582E582850B
:10260B003A82853983F0909003E53B2582F582E58C
:10261B00F0F0053DE53B2408F53BD53C0280030279
:10262B0023E4D082D083D0F0D0E0D0D032C0D0C061
:10263B00E0C0F0C083C08275D0002096030226CC88
:10264B00200E07D53201000228127532FF7809D50A
:10265B003103753108902063E5312582F582E03036
:10266B00E60320E705D8E8022812540790F804F097
:10267B00902200E5312323232582F582AC83AD82A2
:10268B00A3E0F582E5312457F583E0F9AE83AF8201
:10269B000F8E838F82E090F802F00FD9F490F8033D
:1026AB007441F08C838D82E0F8A3EFF0B5000D90B0
:1026BB002063E5312582F582E0C2E7F0C20E0228E5
:1026CB00127532FF90F804E0F5F090F806E090F800
:1026DB0005E020E73B20E53820E62AE5F054072308
:1026EB00239026F07302273C0002271000022710CC
:1026FB000002278B00022710000227100002271070
:10270B00000227100090F8037403F075371EC2B552
:10271B00902200E5312323232582F582E0A3F0905C
:10272B002063E5312582F582E0C2E7F0D20E022864
:10273B0012902200E5312323232582F582AC83AD51
:10274B0082A3E0F582E5312457F583E0F9AE83AF40
:10275B00820F8E838F82E090F802F00FD9F490F8FD
:10276B00037410F08C838D82E0F8A3EFF0B5000DAD
:10277B00902063E5312582F582E0C2E7F002281252
:10278B0090F8037411F02096FD90F804E090F80691
:10279B00E090F805E090F802E0FCE0FD90F803749F
:1027AB0012F0902100E5312323232582F582E030BE
:1027BB00E71DA3E0C082C083F582E531244EF5838B
:1027CB00ECF00582EDF00582E582D083D082F0201B
:1027DB0096FD90F804E090F806E090F805E0BC0256
:1027EB0024902200E5312323232582F582E0A3F0F8
:1027FB00902063E5312582F582E0C2E7F07537035F
:10280B00C2B512281DD20ED082D083D0F0D0E0D02A
:10281B00D02290F8027403F07400F07400F074008E
:10282B00F07411F07400F090F8037441F02096FDF1
:10283B0090F804E0F5F090F806E090F805E0E5F08C
:10284B005407B4011D90F8037410F02096FD90F816
:10285B0004E0F5F090F806E090F805E090F802E05F
:10286B0080DC90F8037411F02096FD90F804E09052
:10287B00F806E090F805E090F802E0E090F80374B9
:10288B0012F02096FD90F804E090F806E090F80521
:10289B00E0227532FF75310890F8037402F0740072
:1028AB00F0740390F809F0747190F805F074879048
:1028BB00F808F0744890F80BF0740090F80CF09056
:1028CB00001212207CF5F0A312207CF58385F08298
:1028DB00E5312582F582E5833400F58312207CF502
:1028EB00F074112582F582E5833400F58312207C88
:1028FB0054E0B4E062902063E5822531F582E5F087
:10290B005407F090F804F090F8027480F07400F023
:10291B00F0F0F0F0F090F8037442F02096FD90F890
:10292B0005E020E52C90F8037411F02096FD90F84B
:10293B0005E090F802E0E090F8037412F02096FDA9
:10294B0090F805E0902063E5822531F582E0D2E630
:10295B00F090F8037401F0D5310302296A01CAD251
:10296B000D7A08902063E5822AF582E030E6405428
:10297B000790F804F090F8027480F07400F0F0F017
:10298B00F0F0F090F8037442F02096FD90F805E01B
:10299B0090F8037411F02096FD90F805E090F80282
:1029AB00E0E090F8037412F02096FD90F805E0DA61
:1029BB00B2C20D753109D20E22C083C0827A0112C8
:1029CB001CC790F7FFA3E582B41002802CB4020C55
:1029DB007A20121CE67A20121CE680E9B4050C7AE8
:1029EB0020121CE67A20121CE680DAB408057AC0A5
:1029FB00121CC7E0122A0980CCD082D08322C0E0FF
:102A0B0003030303122A18D0E0122A1822540F448E
:102A1B0030B43A0040022407FA121CE622060000EA
:102A2B000000000006150000001400040000000068
:102A3B00100E0E04000000000001FF02FF0000005A
:102A4B000006150000000C000C000000000D060035
:102A5B0000003C001E0D4E0D4E0C310C370C3D0C86
:102A6B00430C490CB50D4E0CB50CB80CBE0C4F0CF1
:102A7B005B0C790C7F0C850D4E0C730C610C670C89
:102A8B006D0D4E0D4E0C8B0C910C970C9D0CAF0DD0
:102A9B004E0D4E0D4E0D3C0D4E0CC40CCA0D4E0D75
:102AAB004E0D4E0D4E0CD00CD60CDC0CE20CE80C83
:102ABB00EE0CF40CFA0D000D060D0C0D120D180D8D
:102ACB001E0D240D2A0D300D360D420CA90D481389
:102ADB0044140514880CA30D4E0C550D4E0D4E0DC4
:102AEB004E0D4E0D4E0D4E0D4E0D4E0D4E0D4E0D03
:102AFB004E0D4E0D4E134344205468696E6B52615C
:102B0B00636B2056362E30310D0020434420546821
:102B1B00696E6B5261636B2076362E30312020202C
:102B2B002020200020416C636F726E204D63427237
:102B3B0069646520002053686F7720646174613A83
:102B4B002062616420002053686F77206461746198
:102B5B003A20206F6B200020466C61672042616E2B
:102B6B006B20232031202020466C61672042616E50
:102B7B006B20232032202020466C61672042616E3F
:102B8B006B20232033202020466C61672042616E2E
:102B9B006B2023203420205374617465205661729E
:102BAB006961626C65202357616974696E67206681
:102BBB006F72202020202020202020202020202069
:102BCB00202020202020202020202020202020001A
:102BDB0065787465726E616C2073796E632E2E2E20
:102BEB0020202020202020202020202020202020DA
:102BFB0020202020202020200045787465726E61F3
:102C0B006C2073796E632020202020202020202030
:102C1B0020202020202020202020202020202020A9
:102C2B0020007265636F76657265642E202020200C
:102C3B002020202020202020202020202020202089
:0B2C4B0020202020202020202020003E
:00000001FF
